:0400000017C0FECF58
:10000400FDCFFCCF42C0FACFF9CFF8CF5FC0F6CF17
:10001400F5CFF4CFF3CFF2CFF1CFF0CFEFCFEECFD8
:10002400EDCF01000100060026000000F894EE2741
:10003400ECBBF1E0FBBFEBBFE5BFF8E1F1BDE1BD17
:100044008DE0A2E0BB27ED938A95E9F780E094E088
:10005400A0E6ED930197E9F7E8E2F0E08591959148
:10006400009761F0A591B59105901590BF01F0013D
:1000740005900D920197E1F7FB01F0CFEFE5EDBF9D
:10008400E4E0EEBFC0E6D1E02BC0C0D00A93C3D0F9
:10009400E1E0E51549F47A94772029F45524909801
:1000A400BDD0E4E0E9BF0EC0E0E04599E1E00E2FE9
:1000B400013019F4E0E0E61509F004C0E1E05E2E39
:1000C400E9E07E2E602E0991AED018959FD0A6D07F
:1000D4004A94442019F4909AE0E0E9BFA4D018951A
:1000E40031E041E0EFE3E8BBE0E0E7BBEFE0E5BB94
:1000F400E0E0E4BBE5E0E2BBE1E0E1BBE2E0E3BF7A
:10010400E0E0EFBDE2E0EEBDE0E0EBBDEABDE9BD5D
:10011400E8BDE2BDE2E0E5BDE0E0E4BDE3BDEBBF88
:10012400E5BFE3E0E8B9E0E0E0BF7894E4E6F0E0BE
:100134007FD0E0E08299E1E03E2F303011F441308D
:1001440009F061C0E3B3EF70F0E00E2F1F2FA02F72
:10015400B12FE6E07CD0E07CF3700E2F1F2FE6B3C6
:10016400EF73A02FB12FF0E0EA2BFB2B0E2F1F2FE4
:1001740000951095E02FF12FE130ACEFFA0711F460
:1001840025E037C0E230ACEFFA0711F42FE031C0BC
:10019400E430ACEFFA0711F429E12BC0E830ACEFFE
:1001A400FA0711F423E225C0E031ACEFFA0711F4A9
:1001B4002CE21FC0E032ACEFFA0711F426E319C0B9
:1001C400E034ACEFFA0711F42FE313C0E038ACEFDE
:1001D400FA0711F429E40DC0E030ADEFFA0711F489
:1001E40022E507C0E030AEEFFA0711F42CE501C0B8
:1001F40020E0E0E0E21738F4422E0DD0E0E4E9BF5D
:10020400E4E8F3E015D0432F91CFFFCFEA93FA93BC
:10021400EFB7EA930895E3E8E4BD0895E3E8FFEF58
:10022400FDBDECBD0895E991EFBFF991E991089501
:10023400FA93EA9300C0E991F991309639F08AEF84
:1002440090E00197F1F7A8953197C9F70895EE2347
:100254000E2EFD0121F0EE0FFF1F0A94E1F7089521
:00000001FF
